:10143300C10101E40001E60601E50004E7151D25ED
:011443003573
:101401001214471211D21213E01210A71214617FA5
:081411004078A4E4F608DFFCBA
:0114190022B0
:1013E0007F6443B203E4F5B943B980AE071FEE70E2
:0C13F000FA43B9C0E5B930E5FB43A9029F
:0113FC0022CE
:0414610043EF022231
:1010A700759601759708E59620E7FB75960775977E
:1010B7000FE59620E7FB75960975970FE59620E7EC
:1010C700FB75960B759704E59620E7FB75D7C0432C
:1010D700D72075960F759780E59620E7FB43E602C4
:0110E70022E6
:0E14470043A60CC2A2C2A3E4F5E175E2402266
:1011D200758921758E08758D30758C1575885075D9
:1011E200C80475CADF75CBB175CCDF75CDB1759109
:0E11F200047592DF7593B17594DF7595B12287
:03002B00020003CD
:10000300C0E0C0D075D000C000C2CFD378ECE69476
:100013000018E69400400708E61618700116D00091
:05002300D0D0D0E03256
:1012030053D9BF121401D2AF12145575A4FA75A5A0
:10121300DB75A69643800543902443A06900000034
:101223000000000000000000001209869200120B6B
:031233006C80F6D6
:0C145500759601E4F597E59620E7FB2270
:10004600C290C291C283C282D291E4FF0FBF14FC58
:100056007F3812132C7F3812132CE4FF12132CE472
:10006600FF12132CE4FF12132C7FBA12132C7F23DA
:1000760012132CE4FF12132CE4FF12132CE4FF12CC
:10008600132C7FBA12132C7F2312132C7F431213C7
:100096002C7F4F12132C78E7E6FF12132CE4FF0F88
:1000A600BF14FCC291C282D290E4FF0FBFC8FCC24B
:1000B60093C294C2A7C2A6D294E4FF0FBF14FC7FDA
:1000C600381213597F38121359E4FF121359E4FFFB
:1000D600121359E4FF1213597FBA1213597F2312D0
:1000E6001359E4FF121359E4FF121359E4FF1213D4
:1000F600597FBA1213597F231213597F431213598A
:100106007F4F12135978E8E6FF121359E4FF0FBF29
:1001160014FCC294C2A6D293E4FF0FBFC8FCC296D9
:10012600C297C281C280D297E4FF0FBF14FC7F380A
:100136001213867F38121386E4FF121386E4FF1229
:100146001386E4FF1213867FBA1213867F231213D7
:1001560086E4FF121386E4FF121386E4FF12138669
:100166007FBA1213867F231213867F431213867F6C
:100176004F12138678E9E6FF121386E4FF0FBF14C9
:10018600FCC297C280D296E4FF0FBFC8FCC2A1C2D0
:10019600A2C2A4C2A5D2A2E4FF0FBF14FC7F3812EC
:1001A60013B37F381213B3E4FF1213B3E4FF121331
:1001B600B3E4FF1213B37FBA1213B37F231213B340
:1001C600E4FF1213B3E4FF1213B3E4FF1213B37F79
:1001D600BA1213B37F231213B37F431213B37F4FA5
:1001E6001213B378EAE6FF1213B3E4FF0FBF14FC51
:0601F600C2A2C2A5D2A1C5
:0101FC0022E0
:10132C00E4FEC283E4FD0DBD01FCEF30E704D28284
:10133C008002C282E4FD0DBD01FCD283E4FD0DBD33
:0C134C0002FCEF25E0FF0EBE08D8C283B3
:011358002272
:10135900E4FEC2A7E4FD0DBD01FCEF30E704D2A60F
:101369008002C2A6E4FD0DBD01FCD2A7E4FD0DBDBE
:0C13790002FCEF25E0FF0EBE08D8C2A762
:011385002245
:10138600E4FEC281E4FD0DBD01FCEF30E704D2802E
:101396008002C280E4FD0DBD01FCD281E4FD0DBDDD
:0C13A60002FCEF25E0FF0EBE08D8C2815B
:0113B2002218
:1013B300E4FEC2A4E4FD0DBD01FCEF30E704D2A5B9
:1013C3008002C2A5E4FD0DBD01FCD2A4E4FD0DBD68
:0C13D30002FCEF25E0FF0EBE08D8C2A40B
:0113DF0022EB
:10098600C202E4F508309241C2857F057E0012005E
:100996002E1212687866A6071212687867A60712E2
:1009A60012687868A6071212687869A60712126894
:1009B600786AA607121268786BA607121268786C16
:1009C600A6072092FDD285D2022002090508E50875
:1009D600C3940140B03002247866E630E7107869A7
:1009E600E630E705751C098013751C10800E7869C2
:0E09F600E630E605751C088003751C07A2029A
:010A040022CF
:10126800E4FFFEC283EE25E0FED283E4FD0DBD015E
:10127800FC30820543060180035306FEE4FD0DBDE4
:1012880001FCC283E4FD0DBD02FC0FBF08D7AF0609
:011298002233
:10129900E4FFFEC2A7EE25E0FED2A7E4FD0DBD01E5
:1012A900FC30A60543060180035306FEE4FD0DBD8F
:1012B90001FCC2A7E4FD0DBD02FC0FBF08D7AF06B4
:0112C9002202
:1012CA00E4FFFEC281EE25E0FED281E4FD0DBD0100
:1012DA00FC30800543060180035306FEE4FD0DBD84
:1012EA0001FCC281E4FD0DBD02FC0FBF08D7AF06A9
:0112FA0022D1
:1012FB00E4FFFEC2A4EE25E0FED2A4E4FD0DBD0189
:10130B00FC30A50543060180035306FEE4FD0DBD2D
:10131B0001FCC2A4E4FD0DBD02FC0FBF08D7AF0654
:01132B00229F
:100B6C00E51C24FD602C14603424FD605114605885
:100B7C0014603724F9603D24F0600F24E07055C2F6
:100B8C00AF120F49751C01D2AF22C2AF1203A7D20C
:100B9C00AF22C2AF120D30D2AF751C0422C2AFE42B
:100BAC00FF121020D2AF751C0222300027C2AF12E8
:100BBC000CC6801C30001DC2AF12086180123000C0
:100BCC0013C2AF1206348008300009C2AF1204FD04
:050BDC00D2AFC20022AF
:10102000C2857E4078A4E4F608DEFCE478A4F608E5
:10103000760408A60708760208F608F60876070878
:10104000760108F608760108F6087655F50B750C5A
:1010500000750DA4F50E750F40FB7A00792112067C
:03106000FBD2853B
:01106300226A
:100CC600C2857F4078A4E4F608DFFC78A4760108A4
:100CD60076147866E6FF30E70678A676808004E428
:100CE60078A6F6EF547F78A7F67867E678A8F678C0
:100CF60068E678A9F6786BE678AAF6786CE678ABBB
:100D0600F6796AE778E466601E750B00750C007567
:100D16000DA4750E00750F407B007A00792112062E
:090D2600FB786AE678E4F6D28558
:010D2F0022A1
:10086100C2857F4078A4E4F608DFFC78A47602080C
:1008710076147866E6FF30E70678A676808004E491
:1008810078A6F6EF547F78A7F67867E678A8F67829
:1008910068E678A9F67869E6FF540F78AAF6786ACF
:1008A100E678ABF6786BE6540F79ACF708E678ADED
:1008B100F6EF30E6050876018004E478AEF6786953
:1008C100E678AE30E506E64402F68004E654FDF62D
:1008D10079A7E778E466601E750B00750C00750D4D
:1008E100A4750E00750F407B007A0079211206FB7A
:0808F10078A7E678E4F6D28551
:0108F90022DC
:10063400C202C28578A476030876147866E6FF3091
:10064400E70678A676808004E478A6F6EF547F78EF
:10065400A7F67867E678A8F67868E678A9F6120C23
:100664005692022002030206F87869E630E7030294
:1006740006F578E676067F4078A4E4F608DFFC7495
:10068400524400600978E6E60624A4F876527455CC
:100694004400600978E6E60624A4F87655745844C4
:1006A40000600978E6E60624A4F87658786AE6FF3E
:1006B400600978E6E60624A4F8A607786BE6FF60EE
:1006C4000978E6E60624A4F8A607786CE6FF600934
:1006D40078E6E60624A4F8A607750B00750C0075E9
:1006E4000DA4750E00750F407B007A007921120667
:0606F400FB120A05D2858D
:0106FA0022DD
:1004FD00C28578A476047866E6FE30E70678A6769F
:10050D00808004E478A6F678E6E6B40612EE547F11
:10051D0078A7F67867E678A8F67868E678A9F67988
:10052D00A9E7786866600F78E676067F4078A4E4E0
:10053D00F608DFFC7F407869E6FE543FFD78E466FF
:10054D0070030205D778E6E60624A4F8A605786AB6
:10055D00E6FD78E6E60624A4F8A605786BE6FD78B8
:10056D00E6E60624A4F8A605786CE6FD78E6E60630
:10057D0024A4F8A605EE30E7517869E6543F79E4F6
:10058D00F778E6E6643E7042D20178A5763DE6FF47
:10059D0025E025E0F64401F64402F6750B00750CD6
:1005AD0000750DA4750E00750F407B007A00792142
:1005BD001206FB7869E6543F79E4F778E676067F14
:1005CD004078A4E4F608DFFC7F407869E620E75424
:1005DD00543F78E466604D78A5763DE6FE25E0252E
:1005ED00E0F6300106E64401F6800678A5E654FEF5
:1005FD00F678A5E654FDF6750B00750C00750DA487
:10060D00750E00750F407B007A0079211206FB787C
:10061D0069E6543F79E4F778E676067F4078A4E4FE
:06062D00F608DFFCD28597
:0106330022A4
:100D30007B007A0079341207B5900000E07056FF0E
:100D400074022FF582E43400F583E0FE74E72FF897
:100D5000A60674E72FF8C000E6FE25E0D000F67482
:100D6000E72FF8740146F60FBF04D5E4F5A475A586
:100D7000FF75A60C12004675A4FA75A5DB75A6963C
:100D800043800543902443A0690000000000000058
:050D900000000000005E
:010D9500223B
:100C5600C203E4FFEF75F003A42440F582E43400F8
:100C6600F583E0FE7019EF75F003A42441F582E4E4
:100C76003400F583E0700878E5A607D203803EEEDF
:100C86007867667032EF75F003A42441F582E43488
:100C960000F583E00866701FEF75F003A42442F5A3
:100CA60082E43400F583E0FE08E6543FB50604C24C
:0F0CB60003800AD20380060FEF64147097A20325
:010CC500220C
:100A05007867E6FF78E5E6FE75F003A42440F582F5
:100A1500E43400F583EFF07868E6FFEE75F003A4A3
:100A25002441F582E43400F583EFF008E6543FFFF6
:100A3500EE75F003A42442F582E43400F583EFF06B
:100A450008E6FFEE75F003A42443F582E43400F5CF
:100A550083EFF008E6FFEE75F003A42444F582E485
:100A65003400F583EFF008E6FFEE75F003A42445A6
:0A0A7500F582E43400F583EFF0226F
:10002E0078EBA60608A60743A82078ECE6184670DB
:05003E00F953A8DF22C8
:1012360012010002000000403801380100000000E1
:10124600000109022000010100800F0904000002CC
:101256000000000007058102400005070502024064
:02126600000581
:02144400C104E1
:03004300020EF6B4
:0D0EF600C0E0C0D075D000C005C006C00728
:100F0300759686E59620E7FBAF97759682E5962062
:100F1300E7FBAE97759684E59620E7FBAD97EF3038
:100F2300E203751C40EE30E003751C20EE30E10255
:0B0F3300D204ED30E205D204751C036F
:0B0F3E00D007D006D005D0D0D0E032A4
:100F4900E4FFF508750900750A3FFEAB08050AE5D7
:100F59000AAA097002050914F9E41202430EBE0D2A
:100F6900EAE4F540F541F543F551F54CF54F755077
:100F790040752603F522F523753903F535F53675E0
:090F890096018F97E59620E7FB25
:010F9200223C
:1003A700E4F50875960EF597E59620E7FB759691A7
:1003B700E59620E7FBAF97EF30E411759611759737
:1003C70080E59620E7FBE4F551751C02EF30E2115A
:1003D700759611E4F597E59620E7FBE4F551751C52
:1003E70002EF20E00302049B7B007A00792C7D0852
:1003F7007C00E4FF120D9685310885303185083081
:10040700852F08852E2F85082E853308853233855D
:100417000832E52C54F0248060322480705AE52D90
:1004270014601A24FE601124FA601724FE60182451
:100437000670451210E88043121127803E121161A1
:10044700803912119B8034120028802FE52D24FA61
:10045700601524FE601624FE601724FE601D240C20
:100467007014120AF68014120BE1800F120F93809A
:100477000A12106480058000755102750840E55125
:10048700B40206430820E4F551759611850897E5EF
:100497009620E7FBE4F508E55164017058D3E54E73
:1004A7009440E54D9400500F854E09E4F54DF54E07
:1004B700430808F551800F75094074C0254EF54E65
:1004C70074FF354DF54DE509FD7C00AB52AA53A9E4
:1004D70054E4FF120FDA7E00E5542509F9EE35538F
:1004E700855252F55389544308027596118508972A
:0504F700E59620E7FB83
:0104FC0022DD
:0607B5008B088A09890A85
:1007BB00E4FF75960E1201FDF597E59620E7FB75A4
:1007CB009694E59620E7FBAE97759695E59620E710
:1007DB00FB85970DAB08AA09A90A90000512021612
:1007EB0064036071EE30E60B759614759780E59691
:1007FB0020E7FBEE30E05E759696E59620E7FBAFC3
:10080B0097EF750B00F50C759697E59620E7FBAF08
:10081B0097EFFEEE420BE51CB402087B007A0079E1
:10082B0058800B7400255EF9E43400FA7B01AD0CA3
:10083B00AC0B7F02120D9675960EAB08AA09A90A8E
:10084B001201FDF597E59620E7FB759614E4F597F5
:05085B00E59620E7FB1B
:010860002275
:0606FB008B088A09890A40
:1007010075960E1201FDF597E59620E7FB7596911A
:10071100E59620E7FBAF97759692E59620E7FB8576
:100721009710AB08AA09A90A9000051202166403E2
:1007310070030207B4EF30E50B759611759740E52C
:100741009620E7FBEF20E06BAB08AA09A90A90000D
:1007510001E50E850FF01202AFAB0BAA0CA90DC07B
:1007610003C002C001AB08AA09A90A90000612033E
:100771000CAB08AA09A90A1201FDFF90000112029F
:1007810077FDACF09000061202DC120FDAC3E55CD3
:10079100950FF55CE55B950EF55BE50F2562F5625E
:1007A100E50E3561F561055F759611759701E59661
:0307B10020E7FB43
:0107B4002222
:1010E800E5314530700BE53345327005E540B40213
:1010F800057516028025E4F596852F97E59620E775
:10110800FBE5407007E52F6003754001E540B40139
:0F11180007E52F7003754001E4F5168516512287
:10112700E5334532700DE5406009B40109E5314505
:10113700306003751602E52C541F24FE6004240258
:101147008011E52F452E700BAF31AE30120DF78FA2
:0A115700168003751602851651225A
:10116100E5334532700DE5406009B40109E53145CB
:10117100306003751602E52C541F24FE600424021E
:101181008011E52F452E700BAF31AE30120EA28FBC
:0A1191001680037516028516512220
:10119B00E53145307018E53345327012E540700289
:1011AB00800C901247E493FFE52FD39F40057516F3
:1011BB00028010E52F70057540018007AF2F120ECE
:0711CB004D8F16851651221D
:0100280022B5
:100AF600E52F452E7015E53364024532700DE5404D
:100B06006009B4010BE53145306005751602805267
:100B1600E52C541F14601B14601F2402702FE5314E
:100B2600453060028027E4F556854255E543425537
:100B3600801EE4F555F5568017E4F555F556AF31A8
:100B4600AE3012141ABF030843550180037516020E
:100B5600751601755200755300755455754D00751F
:060B66004E02851651222B
:100BE100E52E24FE6025047062751A00751B12D370
:100BF100E51B9533E51A9532400685321A85331B7C
:100C01007552FF755312755436803D901247E49327
:100C1100FFE52FD39F4005751602802F90124AE4FD
:100C210093F50BA3E493F50A850A1A850B1BD3E50B
:100C31001B9533E51A9532400685321A85331B75AB
:100C410052FF755312755448751601851A4D851B4F
:040C51004E85165165
:010C5500227C
:100F9300E533640145327010E5314530700AE52FC1
:100FA300452E7004E54070057516028020E540B4B7
:100FB300010FE4F555F556F55275530075545580F8
:100FC300097552FF75531275544D751601754D0011
:070FD300754E018516512245
:10106400E52F452E7022E53364014532701AE540C0
:10107400640260028012E54424FFFFE434FFFED3DF
:10108400E5319FE5309E40057516028012755200C9
:1010940075530075544A754D00754E0175160185DA
:0310A400165122C0
:100DF70075968EE59620E7FBAC9775960EEF54EF48
:100E0700F597E59620E7FBEE702DEF24FE6016249C
:100E1700817024759611759710E59620E7FB752666
:100E270003E4FD8014759614759720E59620E7FB7B
:100E3700753903E4FD80027D0275960E8C97E59661
:050E470020E7FBAF05F0
:010E4C002283
:100EA20075968EE59620E7FBAC9775960EEF54EF9C
:100EB200F597E59620E7FBEE702BEF24FE601524F4
:100EC200817022759611759740E59620E7FBE4F54F
:100ED20026FD8013759614759780E59620E7FBE44E
:100EE200F539FD80027D0275960E8C97E59620E716
:030EF200FBAF054E
:010EF50022DA
:10141A00EE7011EF24FE600824817008AD26800664
:08142A00AD3980027D02AF051F
:011432002297
:020E4D008F0A0A
:100E4F00E4F50B7BFF7A1279488B468A47894890E5
:100E5F000005120216650A6005750B028032AB465B
:100E6F00AA47A948900004120216F5447545017B64
:100E7F00007A007949900002E4120255900001E4D3
:100E8F00120255E4120243120A7F754002850A3F8F
:020E9F00AF0B97
:010EA100222E
:100A7F00E4FF75968EE59620E7FBAE979000021285
:100A8F000216705675960E759701E59620E7FB7561
:100A9F0096127597A0E59620E7FBE4F522F523F56E
:100AAF0024752540752181F52675960E759702E5FB
:100ABF009620E7FB759615759780E59620E7FBE482
:100ACF00F535F536F537753840753402F5397596C5
:100ADF000EF597E59630E70480F97F0275960E8E36
:060AEF0097E59620E7FBED
:010AF50022DE
:0A0D96008C0E8D0F8B108A1189124C
:100DA000E50F450E6050EF2420543FF5964396C062
:100DB000E4FFFEE50F24FFFDE50E34FFFCC3EF9DCD
:100DC000EE9C501BE59620E7FBAB10AA11A9128FF1
:100DD000828E83E5971202550FBF00010E80D4E585
:100DE0009620E7FBAB10AA11A9128F828E83E5979C
:060DF000120255E4F59625
:010DF60022DA
:0A0FDA008C118D128B138A148915F7
:100FE400E51245116035EF2420FFE59620E7FBEF7D
:100FF400543FF596E4FFFEC3EF9512EE9511501B96
:10100400AB13AA14A9158F828E83120216F597E5E5
:0B1014009620E7FB0FBF00010E80DC00
:01101F0022AE
:030000000208FAF9
:0C08FA00787FE4F6D8FD7581F302094117
:1001FD00BB010689828A83E0225002E722BBFE0200
:09020D00E32289828A83E4932232
:10021600BB010CE58229F582E5833AF583E022509D
:1002260006E92582F8E622BBFE06E92582F8E222E7
:0D023600E58229F582E5833AF583E4932201
:10024300BB010689828A83F0225002F722BBFE019A
:02025300F32294
:10025500F8BB010DE58229F582E5833AF583E8F0DF
:10026500225006E92582C8F622BBFE05E92582C88B
:02027500F22273
:10027700BB0110E58229F582E5833AF583E0F5F0C5
:10028700A3E0225009E92582F886F008E622BBFEA2
:100297000AE92582F8E2F5F008E222E5832AF583E8
:0802A700E993F5F0A3E99322AD
:1002AF00F8BB0111E58229F582E5833AF583E8F081
:1002BF00E5F0A3F0225009E92582C8F608A6F0223E
:0D02CF00BBFE09E92582C8F2E5F008F22225
:1002DC00BB010DE58229F582E5833AF583020377AC
:1002EC005007E92582F8020365BBFE07E92582F871
:1002FC00020389E58229F582E5833AF58302039BA3
:10030C00BB0120E58229F582E5833AF583D0F0D054
:10031C00E0F8D0E0F9D0E0FAD0E0FBE8C0E0C0F0C3
:10032C000203805018E92582F8D083D082D0E0F9FE
:10033C00D0E0FAD0E0FBC082C08302036EBBFE1893
:10034C00E92582F8D083D082D0E0F9D0E0FAD0E071
:09035C00FBC082C083020392225F
:10090600021203E493A3F8E493A34003F68001F2F2
:1009160008DFF48029E493A3F85407240CC8C333F2
:10092600C4540F4420C8834004F456800146F6DFC1
:10093600E4800B0102040810204080901433E47E0A
:10094600019360BCA3FF543F30E509541FFEE493B6
:10095600A360010ECF54C025E060A840B8E493A37D
:10096600FAE493A3F8E493A3C8C582C8CAC583CAA8
:10097600F0A3C8C582C8CAC583CADFE9DEE780BE60
:0114460000A5
:09036500E6FB08E6FA08E6F922BD
:09036E00EBF608EAF608E9F622B4
:09037700E0FBA3E0FAA3E0F92287
:09038000EBF0A3EAF0A3E9F0227E
:09038900E2FB08E2FA08E2F922A5
:09039200EBF208EAF208E9F2229C
:0C039B00E493FB740193FA740293F922BE
:00000001FF
